Archive member included because of file (symbol)

c:/program files/win-avr/bin/../lib/gcc/avr/4.1.2/avr5\libgcc.a(_exit.o)
                              c:/program files/win-avr/bin/../lib/gcc/avr/4.1.2/../../../../avr/lib/avr5/crtm16.o (exit)
c:/program files/win-avr/bin/../lib/gcc/avr/4.1.2/avr5\libgcc.a(_copy_data.o)
                              Kostka.o (__do_copy_data)
c:/program files/win-avr/bin/../lib/gcc/avr/4.1.2/avr5\libgcc.a(_clear_bss.o)
                              Kostka.o (__do_clear_bss)

Allocating common symbols
Common symbol       size              file

Img                 0x40              Kostka.o

Discarded input sections

 .stabstr       0x00000000        0x0 c:/program files/win-avr/bin/../lib/gcc/avr/4.1.2/../../../../avr/lib/avr5/crtm16.o

Memory Configuration

Name             Origin             Length             Attributes
text             0x00000000         0x00020000         xr
data             0x00800060         0x0000ffa0         rw !x
eeprom           0x00810000         0x00010000         rw !x
*default*        0x00000000         0xffffffff

Linker script and memory map

LOAD c:/program files/win-avr/bin/../lib/gcc/avr/4.1.2/../../../../avr/lib/avr5/crtm16.o
LOAD Kostka.o
LOAD delay.o
LOAD c:/program files/win-avr/bin/../lib/gcc/avr/4.1.2/avr5\libgcc.a
LOAD c:/program files/win-avr/bin/../lib/gcc/avr/4.1.2/../../../../avr/lib/avr5\libc.a
LOAD c:/program files/win-avr/bin/../lib/gcc/avr/4.1.2/avr5\libgcc.a

.hash
 *(.hash)

.dynsym
 *(.dynsym)

.dynstr
 *(.dynstr)

.gnu.version
 *(.gnu.version)

.gnu.version_d
 *(.gnu.version_d)

.gnu.version_r
 *(.gnu.version_r)

.rel.init
 *(.rel.init)

.rela.init
 *(.rela.init)

.rel.text
 *(.rel.text)
 *(.rel.text.*)
 *(.rel.gnu.linkonce.t*)

.rela.text
 *(.rela.text)
 *(.rela.text.*)
 *(.rela.gnu.linkonce.t*)

.rel.fini
 *(.rel.fini)

.rela.fini
 *(.rela.fini)

.rel.rodata
 *(.rel.rodata)
 *(.rel.rodata.*)
 *(.rel.gnu.linkonce.r*)

.rela.rodata
 *(.rela.rodata)
 *(.rela.rodata.*)
 *(.rela.gnu.linkonce.r*)

.rel.data
 *(.rel.data)
 *(.rel.data.*)
 *(.rel.gnu.linkonce.d*)

.rela.data
 *(.rela.data)
 *(.rela.data.*)
 *(.rela.gnu.linkonce.d*)

.rel.ctors
 *(.rel.ctors)

.rela.ctors
 *(.rela.ctors)

.rel.dtors
 *(.rel.dtors)

.rela.dtors
 *(.rela.dtors)

.rel.got
 *(.rel.got)

.rela.got
 *(.rela.got)

.rel.bss
 *(.rel.bss)

.rela.bss
 *(.rela.bss)

.rel.plt
 *(.rel.plt)

.rela.plt
 *(.rela.plt)

.text           0x00000000     0x22aa
 *(.vectors)
 .vectors       0x00000000       0x54 c:/program files/win-avr/bin/../lib/gcc/avr/4.1.2/../../../../avr/lib/avr5/crtm16.o
                0x00000000                __vectors
                0x00000000                __vector_default
 *(.vectors)
 *(.progmem.gcc*)
 *(.progmem*)
 .progmem.data  0x00000054     0x1d74 Kostka.o
                0x00000054                sCube1
                0x00000157                sTime4
                0x00001bb2                Time3
                0x00000199                Cube1
                0x00000198                sTime5
                0x000000d5                sTime2
                0x00000158                sCube5
                0x000000d6                sCube3
                0x00001dc0                Time4
                0x00000116                sTime3
                0x0000181a                Time2
                0x000011d9                Time1
                0x00000095                sCube2
                0x00000117                sCube4
                0x0000121a                Cube2
                0x00001bc0                Cube4
                0x00001832                Cube3
                0x00000094                sTime1
                0x00001dc8                . = ALIGN (0x2)
                0x00001dc8                __trampolines_start = .
 *(.trampolines)
 .trampolines   0x00001dc8        0x0 linker stubs
 *(.trampolines*)
                0x00001dc8                __trampolines_end = .
 *(.jumptables)
 *(.jumptables*)
 *(.lowtext)
 *(.lowtext*)
                0x00001dc8                __ctors_start = .
 *(.ctors)
                0x00001dc8                __ctors_end = .
                0x00001dc8                __dtors_start = .
 *(.dtors)
                0x00001dc8                __dtors_end = .
 SORT(*)(.ctors)
 SORT(*)(.dtors)
 *(.init0)
 .init0         0x00001dc8        0x0 c:/program files/win-avr/bin/../lib/gcc/avr/4.1.2/../../../../avr/lib/avr5/crtm16.o
                0x00001dc8                __init
 *(.init0)
 *(.init1)
 *(.init1)
 *(.init2)
 .init2         0x00001dc8        0xc c:/program files/win-avr/bin/../lib/gcc/avr/4.1.2/../../../../avr/lib/avr5/crtm16.o
 *(.init2)
 *(.init3)
 *(.init3)
 *(.init4)
 .init4         0x00001dd4       0x16 c:/program files/win-avr/bin/../lib/gcc/avr/4.1.2/avr5\libgcc.a(_copy_data.o)
                0x00001dd4                __do_copy_data
 .init4         0x00001dea       0x10 c:/program files/win-avr/bin/../lib/gcc/avr/4.1.2/avr5\libgcc.a(_clear_bss.o)
                0x00001dea                __do_clear_bss
 *(.init4)
 *(.init5)
 *(.init5)
 *(.init6)
 *(.init6)
 *(.init7)
 *(.init7)
 *(.init8)
 *(.init8)
 *(.init9)
 .init9         0x00001dfa        0x8 c:/program files/win-avr/bin/../lib/gcc/avr/4.1.2/../../../../avr/lib/avr5/crtm16.o
 *(.init9)
 *(.text)
 .text          0x00001e02        0x4 c:/program files/win-avr/bin/../lib/gcc/avr/4.1.2/../../../../avr/lib/avr5/crtm16.o
                0x00001e02                __vector_1
                0x00001e02                __vector_12
                0x00001e02                __bad_interrupt
                0x00001e02                __vector_6
                0x00001e02                __vector_3
                0x00001e02                __vector_11
                0x00001e02                __vector_13
                0x00001e02                __vector_17
                0x00001e02                __vector_7
                0x00001e02                __vector_5
                0x00001e02                __vector_4
                0x00001e02                __vector_9
                0x00001e02                __vector_2
                0x00001e02                __vector_15
                0x00001e02                __vector_8
                0x00001e02                __vector_14
                0x00001e02                __vector_10
                0x00001e02                __vector_16
                0x00001e02                __vector_18
                0x00001e02                __vector_20
 .text          0x00001e06      0x450 Kostka.o
                0x00001e06                changeImg
                0x00001f50                __vector_19
                0x00002098                main
 .text          0x00002256       0x52 delay.o
                0x00002256                delayloop32
 .text          0x000022a8        0x0 c:/program files/win-avr/bin/../lib/gcc/avr/4.1.2/avr5\libgcc.a(_exit.o)
 .text          0x000022a8        0x0 c:/program files/win-avr/bin/../lib/gcc/avr/4.1.2/avr5\libgcc.a(_copy_data.o)
 .text          0x000022a8        0x0 c:/program files/win-avr/bin/../lib/gcc/avr/4.1.2/avr5\libgcc.a(_clear_bss.o)
                0x000022a8                . = ALIGN (0x2)
 *(.text.*)
 .text.libgcc   0x000022a8        0x0 c:/program files/win-avr/bin/../lib/gcc/avr/4.1.2/avr5\libgcc.a(_exit.o)
 .text.libgcc   0x000022a8        0x0 c:/program files/win-avr/bin/../lib/gcc/avr/4.1.2/avr5\libgcc.a(_copy_data.o)
 .text.libgcc   0x000022a8        0x0 c:/program files/win-avr/bin/../lib/gcc/avr/4.1.2/avr5\libgcc.a(_clear_bss.o)
                0x000022a8                . = ALIGN (0x2)
 *(.fini9)
 .fini9         0x000022a8        0x0 c:/program files/win-avr/bin/../lib/gcc/avr/4.1.2/avr5\libgcc.a(_exit.o)
                0x000022a8                exit
                0x000022a8                _exit
 *(.fini9)
 *(.fini8)
 *(.fini8)
 *(.fini7)
 *(.fini7)
 *(.fini6)
 *(.fini6)
 *(.fini5)
 *(.fini5)
 *(.fini4)
 *(.fini4)
 *(.fini3)
 *(.fini3)
 *(.fini2)
 *(.fini2)
 *(.fini1)
 *(.fini1)
 *(.fini0)
 .fini0         0x000022a8        0x2 c:/program files/win-avr/bin/../lib/gcc/avr/4.1.2/avr5\libgcc.a(_exit.o)
 *(.fini0)
                0x000022aa                _etext = .

.data           0x00800060       0x36 load address 0x000022aa
                0x00800060                PROVIDE (__data_start, .)
 *(.data)
 .data          0x00800060        0x0 c:/program files/win-avr/bin/../lib/gcc/avr/4.1.2/../../../../avr/lib/avr5/crtm16.o
 .data          0x00800060       0x36 Kostka.o
                0x00800060                Data
 .data          0x00800096        0x0 delay.o
 .data          0x00800096        0x0 c:/program files/win-avr/bin/../lib/gcc/avr/4.1.2/avr5\libgcc.a(_exit.o)
 .data          0x00800096        0x0 c:/program files/win-avr/bin/../lib/gcc/avr/4.1.2/avr5\libgcc.a(_copy_data.o)
 .data          0x00800096        0x0 c:/program files/win-avr/bin/../lib/gcc/avr/4.1.2/avr5\libgcc.a(_clear_bss.o)
 *(.data*)
 *(.rodata)
 *(.rodata*)
 *(.gnu.linkonce.d*)
                0x00800096                . = ALIGN (0x2)
                0x00800096                _edata = .
                0x00800096                PROVIDE (__data_end, .)

.bss            0x00800096       0x46
                0x00800096                PROVIDE (__bss_start, .)
 *(.bss)
 .bss           0x00800096        0x0 c:/program files/win-avr/bin/../lib/gcc/avr/4.1.2/../../../../avr/lib/avr5/crtm16.o
 .bss           0x00800096        0x6 Kostka.o
                0x00800099                currentViz
                0x00800097                currentY
                0x00800098                currentImg
                0x0080009a                zmena
                0x0080009b                time
                0x00800096                currentX
 .bss           0x0080009c        0x0 delay.o
 .bss           0x0080009c        0x0 c:/program files/win-avr/bin/../lib/gcc/avr/4.1.2/avr5\libgcc.a(_exit.o)
 .bss           0x0080009c        0x0 c:/program files/win-avr/bin/../lib/gcc/avr/4.1.2/avr5\libgcc.a(_copy_data.o)
 .bss           0x0080009c        0x0 c:/program files/win-avr/bin/../lib/gcc/avr/4.1.2/avr5\libgcc.a(_clear_bss.o)
 *(.bss*)
 *(COMMON)
 COMMON         0x0080009c       0x40 Kostka.o
                0x0080009c                Img
                0x008000dc                PROVIDE (__bss_end, .)
                0x000022aa                __data_load_start = LOADADDR (.data)
                0x000022e0                __data_load_end = (__data_load_start + SIZEOF (.data))

.noinit         0x008000dc        0x0
                0x008000dc                PROVIDE (__noinit_start, .)
 *(.noinit*)
                0x008000dc                PROVIDE (__noinit_end, .)
                0x008000dc                _end = .
                0x008000dc                PROVIDE (__heap_start, .)

.eeprom         0x00810000        0x0
 *(.eeprom*)
                0x00810000                __eeprom_end = .

.stab           0x00000000      0x378
 *(.stab)
 .stab          0x00000000      0x378 c:/program files/win-avr/bin/../lib/gcc/avr/4.1.2/../../../../avr/lib/avr5/crtm16.o

.stabstr        0x00000000       0x71
 *(.stabstr)
 .stabstr       0x00000000       0x71 c:/program files/win-avr/bin/../lib/gcc/avr/4.1.2/../../../../avr/lib/avr5/crtm16.o

.stab.excl
 *(.stab.excl)

.stab.exclstr
 *(.stab.exclstr)

.stab.index
 *(.stab.index)

.stab.indexstr
 *(.stab.indexstr)

.comment
 *(.comment)

.debug
 *(.debug)

.line
 *(.line)

.debug_srcinfo
 *(.debug_srcinfo)

.debug_sfnames
 *(.debug_sfnames)

.debug_aranges  0x00000000       0x40
 *(.debug_aranges)
 .debug_aranges
                0x00000000       0x20 Kostka.o
 .debug_aranges
                0x00000020       0x20 delay.o

.debug_pubnames
                0x00000000      0x175
 *(.debug_pubnames)
 .debug_pubnames
                0x00000000      0x153 Kostka.o
 .debug_pubnames
                0x00000153       0x22 delay.o

.debug_info     0x00000000      0x805
 *(.debug_info)
 .debug_info    0x00000000      0x6c5 Kostka.o
 .debug_info    0x000006c5      0x140 delay.o
 *(.gnu.linkonce.wi.*)

.debug_abbrev   0x00000000      0x173
 *(.debug_abbrev)
 .debug_abbrev  0x00000000      0x123 Kostka.o
 .debug_abbrev  0x00000123       0x50 delay.o

.debug_line     0x00000000      0x431
 *(.debug_line)
 .debug_line    0x00000000      0x38a Kostka.o
 .debug_line    0x0000038a       0xa7 delay.o

.debug_frame    0x00000000       0x70
 *(.debug_frame)
 .debug_frame   0x00000000       0x50 Kostka.o
 .debug_frame   0x00000050       0x20 delay.o

.debug_str      0x00000000       0x3a
 *(.debug_str)
 .debug_str     0x00000000       0x3a Kostka.o

.debug_loc
 *(.debug_loc)

.debug_macinfo
 *(.debug_macinfo)
OUTPUT(Kostka.elf elf32-avr)
LOAD linker stubs
